:100000000C945D000C9485000C9485000C94850084
:100010000C9485000C9485000C9485000C9485004C
:100020000C9485000C9485000C9485000C9485003C
:100030000C9485000C9485000C9485000C9485002C
:100040000C9462030C9485000C9430030C940A0306
:100050000C9485000C9485000C9485000C9485000C
:100060000C9485000C9485000000000024002700FB
:100070002A0000000000250028002B0004040404CE
:100080000404040402020202020203030303030342
:10009000010204081020408001020408102001021F
:1000A00004081020000000080002010000030407FB
:1000B0000000000000000000AC0311241FBECFEFC1
:1000C000D8E0DEBFCDBF11E0A0E0B1E0E6E4FBE0A8
:1000D00002C005900D92A433B107D9F722E0A4E342
:1000E000B1E001C01D92A435B207E1F710E0CDE503
:1000F000D0E004C02197FE010E948105CC35D107D4
:10010000C9F70E94EB030C94A1050C940000E1EBED
:10011000F0E02491EDE9F0E09491E9E8F0E0E49179
:10012000EE23C9F0222339F0233001F1A8F4213065
:1001300019F1223029F1F0E0EE0FFF1FEE58FF4FCA
:10014000A591B4912FB7F894EC91811126C09095A8
:100150009E239C932FBF08952730A9F02830C9F023
:10016000243049F7209180002F7D03C0209180002A
:100170002F7720938000DFCF24B52F7724BDDBCFEE
:1001800024B52F7DFBCF2091B0002F772093B000B6
:10019000D2CF2091B0002F7DF9CF9E2BDACFAF9236
:1001A000BF92CF92DF92EF92FF920F931F93CF9364
:1001B000DF936C017B018B01040F151FEB015E01C6
:1001C000AE18BF08C017D10759F06991D601ED915B
:1001D000FC910190F081E02DC6010995892B79F7FA
:1001E000C501DF91CF911F910F91FF90EF90DF90AC
:1001F000CF90BF90AF900895FC01538D448D252F73
:1002000030E0842F90E0821B930B541710F0CF96B0
:10021000089501970895FC01918D828D981761F0E2
:10022000A28DAE0FBF2FB11D5D968C91928D9F5FF9
:100230009F73928F90E008958FEF9FEF0895FC01D8
:10024000918D828D981731F0828DE80FF11D858D8B
:1002500090E008958FEF9FEF0895FC01918D228D1E
:10026000892F90E0805C9F4F821B91098F739927A3
:10027000089589E491E00E942D0121E0892B09F481
:1002800020E0822F089580E090E0892B29F00E94E1
:10029000390181110C9400000895FC01A48DA80F70
:1002A000B92FB11DA35ABF4F2C91848D90E00196B8
:1002B0008F739927848FA689B7892C93A089B189D8
:1002C0008C91837080648C93938D848D981306C079
:1002D0000288F389E02D80818F7D80830895EF92DD
:1002E000FF920F931F93CF93DF93EC0181E0888FF0
:1002F0009B8D8C8D98131AC0E889F989808185FFC0
:1003000015C09FB7F894EE89FF896083E889F98961
:1003100080818370806480839FBF81E090E0DF9163
:10032000CF911F910F91FF90EF900895F62E0B8DB6
:1003300010E00F5F1F4F0F731127E02E8C8D8E1171
:100340000CC00FB607FCFACFE889F989808185FFD8
:10035000F5CFCE010E944D01F1CFEB8DEC0FFD2FBB
:10036000F11DE35AFF4FF0829FB7F8940B8FEA8993
:10037000FB8980818062CFCFCF93DF93EC01888DA2
:100380008823B9F0AA89BB89E889F9898C9185FD10
:1003900003C0808186FD0DC00FB607FCF7CF8C919E
:1003A00085FFF2CF808185FFEDCFCE010E944D0108
:1003B000E9CFDF91CF9108953FB7F894809139014B
:1003C00090913A01A0913B01B0913C0126B5A89BC8
:1003D00005C02F3F19F00196A11DB11D3FBFBA2FD7
:1003E000A92F982F8827BC01CD01620F711D811D97
:1003F000911D42E0660F771F881F991F4A95D1F71C
:100400000895AF92BF92CF92DF92EF92FF920F9337
:100410001F93CF93DF938B01D0E0C0E001975C0185
:1004200080914A0290914B02DC01ED91FC91008495
:10043000F185E02D0995A816B906ACF00E94DC0103
:100440006B017C010E94DC016C197D098E099F09FA
:10045000683E734081059105A8F321960C171D078E
:10046000F9F680E001C081E0DF91CF911F910F91FB
:10047000FF90EF90DF90CF90BF90AF900895DC0198
:10048000ED91FC910190F081E02D0994CF92DF92E3
:10049000EF92FF920F931F93CF93DF9300D000D082
:1004A000CDB7DEB78C01FC0101900020E9F7319750
:1004B000E81BF90B86E080933D01E0933E0110922A
:1004C0003F011092400180913D0190913E01A09129
:1004D0003F01B091400189839A83AB83BC836CEF69
:1004E0007FEF80914A0290914B020E943F02CE0121
:1004F00001967C016E0195E0C90ED11C80914A02E3
:1005000090914B02D7016D917D01DC01ED91FC9141
:100510000190F081E02D0995EC14FD0479F76DEF61
:100520007FEF80914A0290914B020E943F026EEF52
:100530007FEF80914A0290914B020E943F02F12C82
:100540002F2D30E0F80101900020E9F73197E01BF2
:10055000F10B80914A0290914B022E173F0758F4FD
:10056000200F311FF9016081062E000C770B0E94CD
:100570003F02F394E5CF6FEF7FEF0F900F900F9056
:100580000F90DF91CF911F910F91FF90EF90DF902F
:10059000CF900C943F020F931F93CF93DF93CDB76F
:1005A000DEB764970FB6F894DEBF0FBECDBF8C01E7
:1005B00062E171E00E948705892B69F481E00E9465
:1005C000870065E171E0CE0101960E949A05CE0197
:1005D00001960E94460262E271E0C8010E9487050E
:1005E000892B69F480E00E94870066E271E0CE0109
:1005F00001960E949A05CE0101960E9446026496D9
:100600000FB6F894DEBF0FBECDBFDF91CF911F9123
:100610000F9108951F920F920FB60F9211242F93EE
:100620003F934F935F936F937F938F939F93AF937A
:10063000BF93EF93FF9389E491E00E944D01FF91F6
:10064000EF91BF91AF919F918F917F916F915F914A
:100650004F913F912F910F900FBE0F901F901895C3
:100660001F920F920FB60F9211242F938F939F9387
:10067000EF93FF93E0915901F0915A018081E0914D
:100680005F01F091600182FD1BC090818091620149
:100690008F5F8F7320916301821741F0E0916201B7
:1006A000F0E0E75BFE4F958F80936201FF91EF9141
:1006B0009F918F912F910F900FBE0F901F901895C3
:1006C0008081F4CF1F920F920FB60F9211242F93B7
:1006D0003F938F939F93AF93BF93809135019091F8
:1006E0003601A0913701B09138013091340123E0F7
:1006F000230F2D3758F50196A11DB11D209334010C
:100700008093350190933601A0933701B09338015F
:100710008091390190913A01A0913B01B0913C0147
:100720000196A11DB11D8093390190933A01A093C8
:100730003B01B0933C01BF91AF919F918F913F914D
:100740002F910F900FBE0F901F90189526E8230F42
:100750000296A11DB11DD2CFE9E4F1E0138212820D
:1007600088EE93E0A0E0B0E084839583A683B7830E
:1007700084E091E09183808385EC90E09587848785
:1007800084EC90E09787868780EC90E0918B808B5B
:1007900081EC90E0938B828B82EC90E0958B848B44
:1007A00086EC90E0978B868B118E128E138E148EB2
:1007B000F0934B02E0934A02E1E4F1E089E980839F
:1007C00087E1818384E3828381E0838314821582BD
:1007D000168217820895CF93DF93CDB7DEB72C979B
:1007E0000FB6F894DEBF0FBECDBF789484B582609B
:1007F00084BD84B5816084BD85B5826085BD85B5C5
:10080000816085BD80916E00816080936E00109242
:1008100081008091810082608093810080918100BD
:10082000816080938100809180008160809380004E
:100830008091B10084608093B1008091B0008160AC
:100840008093B00080917A00846080937A008091D8
:100850007A00826080937A0080917A008160809330
:100860007A0080917A00806880937A001092C100AB
:10087000EDE9F0E02491E9E8F0E08491882399F033
:1008800090E0880F991FFC01E859FF4FA591B491A2
:10089000FC01EE58FF4F859194918FB7F894EC913D
:1008A000E22BEC938FBFE0915901F0915A0182E065
:1008B0008083E0915901F0915A011082E091550135
:1008C000F09156011082E0915701F091580180E1BA
:1008D000808310926101E0915D01F0915E0186E0FC
:1008E0008083E0915B01F0915C0180818061808375
:1008F000E0915B01F0915C01808188608083E091F0
:100900005B01F0915C01808180688083E0915B01F4
:10091000F0915C0180818F7D8083809145018860AA
:10092000809345018BEC92E09093530280935202A6
:100930006E018DE0C80ED11C90E0E92E90E0F92EFA
:1009400080914A0290914B02DC01ED91FC91008470
:10095000F185E02D0995892B09F450C080914A0258
:1009600090914B02DC01ED91FC910284F385E02D26
:1009700009958C3F09F042C064E670E085E090E0A4
:100980000E9401028823D1F18E01075F1F4F580199
:1009900080914A0290914B02DC01ED91FC9102841E
:1009A000F385E02D0995F80181938F01EC15FD0584
:1009B00079F780914A0290914B02DC01ED91FC9114
:1009C0000284F385E02D099589853A852B859C85E0
:1009D00080933D0130933E0120933F01909340016D
:1009E000833009F476C0B0F4813009F446C0E09158
:1009F0004C02F0914D02823009F46FC0E114F10411
:100A000009F49ECF0E943901882309F499CF0E94EE
:100A1000000096CF843009F462C0853079F7809069
:100A20003E01082D10E062E370E0C80102960E94CA
:100A30000102882319F380914A0290914B02DC0154
:100A4000ED91FC910284F385E02D099586EEA82EA8
:100A500081E0B82E912C80914A0290914B02DC01EA
:100A6000ED91FC910284F385E02D8914E9F109955B
:100A7000F50181935F019394EECF88E0E1E4F1E02A
:100A8000DE01119601900D928A95E1F76EEF7FEFEE
:100A900080914A0290914B020E943F028E010F5FAB
:100AA0001F4FF80161918F01062E000C770B80918A
:100AB0004A0290914B020E943F02A016B10689F7AC
:100AC0006FEF7FEF80914A0290914B020E943F02AC
:100AD00095CFE0914E02F0914F0209958FCFE091B2
:100AE0005002F0915102F9CF0995F801EA51FE4FF9
:100AF0001082E0915202F091530286EE91E0099546
:100B00007DCFEE0FFF1F0590F491E02D0994FB01BE
:100B1000DC018D9181341CF08B350CF4805E619189
:100B200061341CF06B350CF4605E861B611189F337
:100B3000990B0895FB01DC0101900D920020E1F773
:060B40000895F894FFCFB8
:100B4600000000006F01CF00FC00BC012D010B016D
:100B56001F014F4E007B224C6564223A224F6E22C3
:100B66007D004F4646007B224C6564223A224F6642
:040B760066227D0076
:00000001FF
